:030000000219FDE5
:03000B000200AA46
:03002B0002015F70
:03005B000202F5A9
:030073000202DBAB
:1000800002030406080C10182030406080040608A3
:100090000C10182030406080A0C000070F1F3F0DDB
:1000A0000D0403060D0502030202C2AFC0D0C0E07A
:1000B000206217E5256002E473E525F4F58A758B67
:1000C00000D262D0E0D0D0D2AF3285268AC262E5BB
:1000D00026F4602F758B00D0E0D0D0C297C295C2B5
:1000E00093D2AF32C297C295C293206E0C2066099C
:1000F000740ED5E0FDE57E4290758B00D0E0D0D047
:10010000D2AF32758A00C28DD26201F901B930686E
:1001100005206602D29701B9306805206602D295A3
:1001200001B9306805206602D29301B9C2963068E1
:100130000A206607740CD5E0FDD29701B9C294304D
:10014000680A206607740CD5E0FDD29501B9C29209
:1001500030680A206607740CD5E0FDD29301B9C25D
:10016000AFC2AD53E6EFC0D0C0E0D2D3D2AFC2CE63
:10017000E52A6007207449152A21C07800790020FB
:10018000742EE580307E01F430E30278FF53DACF3D
:10019000207E0343DA20307E0343DA10C2D8C271D6
:1001A000E580307E01F430E30279FFC3E89970CB3B
:1001B000306103752A40207403752A40885FD2702D
:1001C00020740DE52B6004152B21D043DA01C2D831
:1001D00020700221E3A85F206102C2702074022116
:1001E000E188227882B60403852224C3E525944061
:1001F0004002D26420CF0AD0E0D0D043E610D2AD86
:1002000032C2CF053A7802E52A6005307402152A19
:10021000C3E55F94014005756200412D756300756B
:100220006C00E5622401F56250037562FF7982B7C4
:10023000020D306D1DC3E52294324016854D2279A2
:1002400082B7030E306D0BC3E52294324004798EE1
:100250008722C3E5239522600840041523416105E8
:1002600023D8CA056CE56C7002156CD56D63756D8D
:10027000017805C3E56C956E4057C3E56C956F50EA
:10028000087801756D03020295C3E56C9570500501
:100290007801756D01C3E5659524401E7982B70428
:1002A0000241C6206D14852465E56C046003856EEB
:1002B0006C756D0175233C0202D1E565285005750A
:1002C00065FF41C6F565E5650470067563FF756CED
:1002D000FFD0E0D0D043E610D2AD32C2AFC0D05391
:1002E000E67FC26075910085569485579575910497
:1002F000D0D0D2AF32C2AF53E6EFC2ADC0D0C0E073
:10030000C0F0D2D3D2AFA8FBA9FCC2D83071026131
:100310005C53DACF207E0343DA10307E0343DA20C9
:10032000D271E580307E01F420E3026133882789B1
:1003300028A13B53DACF207E0343DA20307E0343EB
:10034000DA10C2D8C271307402A1277800E580307B
:100350007E01F430E302A127885FA10F53DACF209A
:100360007E0343DA20307E0343DA10C2712061023B
:10037000813553DACF207E0343DA10307E0343DA2F
:1003800020C2D8D271885A895BC3E89558F8E9959C
:1003900059F97B007E087A00C3E8948CE9940050F8
:1003A00005755E008127882178A2E6A8216055C3E3
:1003B000E894C8E994005008E4D2E4FB7A0A810288
:1003C000C3E89468E994015008E4D2E3FB7A0F8112
:1003D00002C3E894D0E994025008E4D2E2FB7A1E0A
:1003E0008102C3E894A0E994055008E4D2E1FB7AC5
:1003F0003C8102C3E89498E994085008E4D2E0FBF9
:100400007A787E00C3E8955CFCE9955DFD30E70AEB
:10041000ECF42401FCEDF43400FD755E00C3EC9AAD
:10042000ED9E5003755E01885C895D855A58855B39
:10043000597802A10FC3E89527F8E99528F9307C8F
:100440000281F3307B0281F3307A0281EC20750265
:100450008158E9FDE8FC8177E9C313F9E813F83026
:10046000790281ECE9C313F9E813F830780281ECE2
:0F047000E9C313FDE813FC206126C3EC941CEDD7
:10047F0094024002818EED7018C3EC94C85012059F
:10048F0029C3E529940A5002A127755F00D270A1F4
:10049F0027E529600215297400207F037896E6244A
:1004AF00FAFEE43400FFC3EC9EFCED9FFD5006788E
:1004BF0000790081F3C3EC94FFED9400400678FFC0
:1004CF00790081F3EC8575F0A4C5F0A2F733F879C4
:1004DF0000400302050F78FF790002050FE9C313EF
:1004EF00F9E813F8307C0EE9600278FFC3E813389F
:1004FF00F8E43400F9C3E894FFE99400400278FF70
:10050F00885FD270206102A127741FF4552F4BF51D
:10051F002FC274EB7002D274752A40307403752A9F
:10052F000A306102A13B20740353DAFE2074037575
:10053F002B20D0F0D0E0D0D0D2AD43E610327901ED
:10054F0002056B790302056B790A02056B791E02AE
:10055F00056B796402056B79C802056B7817E4D5D2
:10056F00E0FDD8FAD9F6227A147B780205927A1038
:10057F007B8C0205927A0D7BB40205927A0B7BC8B5
:10058F000205927902B27DE4C294D5E0FDD295D5F1
:10059F00E0FDC295D5E0FDD294D5E0FDD297E5768A
:1005AF00D5E0FDC2977496D5E0FDD9D9EAF8D5E02C
:1005BF00FDD8FBDBCEC29422C37C007D0075F0001A
:1005CF0005F0EA33FAEB33FB50F6EB13FBEA13FAC1
:1005DF00C3E9FFE8FEE89AF8E99BF95004EFF9EE5A
:1005EF00F8B3EC33FCED33FDD5F0DFEDF9ECF82289
:1005FF00E889F08A20D2D4F8A9F07B0030F70B7B82
:10060F00FFF42401F8E9F43400F9E88520F0A4ADF3
:10061F00F0F8E98520F0A4AFF0FEED2EF974003F5D
:10062F00FA7C04C3EA13FAE913F9E813F8DCF48B44
:10063F00F030F70AE8F42401F8E9F43400F9E88916
:10064F00F0C2D4F8A9F0227882B604030206F5C3EB
:10065F00E55F9419401EE52D54067018206D36780D
:10066F00057994E7146007780A1460027812C3E5DD
:10067F004198401F306D09856765756CFF756D0179
:10068F00852224E4F545F546F547F548F549C26D51
:10069F000206F5D26D7994E7147013E523F4333322
:1006AF00F913F8E9540104F9E854FE0206E9E714D6
:1006BF00147014E523F4333333F913F8E9540304B6
:1006CF00F9E854FC0206F1E523F433333333F9131D
:1006DF00F8E954070404F9E854F8C39440F8E9948E
:1006EF0000F98845894622C3E54113F9E54013F81F
:1006FF00C3E54598F8E54699F9500CC3E89480E9AD
:10070F0094FF401602072DC3E8947FE9940050032D
:10071F0002072D787F790002072D788079FF884AAC
:10072F00894B22E54A2547F8E54B3548F9854B209B
:10073F00E4300701F43549FA30E709C3EA94F04091
:10074F001502076BC3EA940F500302076B78FF790A
:10075F00FF7A0F02076B780079007AF0C3E52495D2
:10076F0064500AC374019524500B020789E54B208E
:10077F00E70E020789E54B30E706884789488A4923
:10078F002278A4E6FAC3E54A33F8E54B33F9B1FF13
:10079F00E930E70BC3E89480E994FF4013E1C3C34A
:1007AF00E8947FE994005002E1C3787F7900E1C3B8
:1007BF00788079FFE820E715C3E52398F84009C34F
:1007CF00E8940140030207EA78010207EAE8F424FB
:1007DF00012523F840030207EA78FF884C2278A509
:1007EF00E6FAA848A949B1FFE930E70CC3E894013C
:1007FF00E994FF401602081EC3E894FFE9940050E5
:10080F000302081E78FF790002081E780179FFE9BC
:10081F0020E715C3E54C98F84009C3E8940140035D
:10082F000208457801020845E8F42401254CF840F8
:10083F000302084578FF88242278FFC26420693DAF
:10084F00206A12D264C3E541940A4009C3E5259496
:10085F00405002C26479A1E76023E541601F74FF35
:0F086F008541F0848539F0306A0375F005A4F8EF
:10087E00C5F0600278FFC3E895675002A8678866E6
:10088E0022C3E5409440E5419401E566500314010E
:10089E00A0046002F566227883E6F520120F5975E2
:1008AE00E89012054D75E890E5E820ECFBA8BDA98F
:1008BE00BE120FF3757130757200C3740013FD74A0
:1008CE0030606613FC74302CFC74003DFDECFAEDC8
:1008DE00FBC3E89AE99B4014E5712430F571E5728B
:1008EE003400F572EA2CFAEB3DFB80E5AE71AF7287
:1008FE00C3E57213F9E57113F8C3E913F9E813F8B8
:10090E007A03C3E913F9E813F8DAF7AA201A700983
:10091E007571007572000209371AEA6008EE28FE3A
:10092E00EF39FFDAF88E718F722275E89022788394
:10093E00E6FFE5E820ECF7A8BDA9BE0573C3E57395
:10094E0094084052757300E9FA79A0E76044EA70A2
:10095E0007E574601B020972C3E895746010E574B4
:10096E005006600C1402097E0460F902097EE574DB
:10097E00F574C394A8401B7564C0C39405401375E9
:10098E006480C39405400B756440C39405400375A1
:10099E00640075BB0122EFC39401601F7430601BAD
:1009AE00C3E894FFE994035012C3E89571E9957278
:1009BE005009E564600C15640209D0E564F4600228
:1009CE000564A864C3E524985002A824C3E895657D
:1009DE00400AA865E565F460038565648825882668
:1009EE00E573B4070375BB1E22743279A687F0A493
:1009FE00C5F0A2F733F8C3E895644002A8648822D4
:100A0E008824882588268867227540007541F02243
:100A1E00C2AF75C820A8CCA9CDAA3A30CF010A75AD
:100A2E00C824D2AFAB3BAC3C883B893CC3E89BF8B7
:100A3E00E99C206908F930670261334190AD3D8A27
:100A4E003DF9EA9DFA600478FF79FFAE3EAF3F8B29
:100A5E003E8C3FC3EC9FFCC3E99CF542A83BA93CEE
:100A6E00C3E89EF8E99FF9C3E54113FBE54013FA8D
:100A7E00E82AF540E93BF54150067540FF7541FF08
:100A8E0041DAAA40AB41AC40AD417E047F02C3EBDC
:100A9E00940440021E1FC3EB940840021E1FC3EDB8
:100AAE0013FDEC13FCDEF7C3EA9CFAEB9DFBEF6043
:100ABE0009C3E913F9E813F8DFF7EA28FAEB39FB73
:100ACE008A408B4150067BFF8B408B41C3EB9402D7
:100ADE005002D2673069047F0361057892E6FFC346
:100AEE00E537948240110FC3E53794A040010FC340
:100AFE00EF940640027F057E06E541C4540FF9E5EA
:100B0E0041C454F0F8E540C4540F28F8C3E89EFAE7
:100B1E00E99400FB4009C3EA9402EB940050047A76
:100B2E0002E4FB617FAA40AB41EBC4FEEAC4540F62
:100B3E004EFCC3EA9CFAEB9400FBC3E813C313F814
:100B4E00EA28FAEB3400FB8A408B41C3EB94024057
:100B5E0002C2677806EBC4FE7B00EAC4540F4EFA5D
:100B6E00C3EA98FA4005C3940250027A027892E6DC
:100B7E00FF306002617F855256855357D26043E63F
:100B8E0080C3E49AF8E49BF93067028119E8FAE928
:100B9E00FBD3E913FDE813FC88528953C3EF94038A
:100BAE006038EF20E00DE82CF8E93DF9ECFAEDFBAA
:100BBE00020BD4E828F8E939F9C3E82402F8E9343D
:100BCE0000F97AFE7BFFC3EF9403400E8A548B55D7
:100BDE00884E894F8C508D51814D885489558A4E3F
:100BEE008B4F8C508D51306920C3E53394034019DF
:100BFE00E542A2E713F8E555F4240138400B20E74F
:100C0E00087554FFF42401F555814DE8FAD3E81325
:100C1E00FC8852C3EF94036020EF20E007E82CF825
:100C2E00ECFA8139E8282402F87AFEC3EF940340E7
:100C3E00088A54884E8C50814D88548A4E8C50E5CB
:100C4E006BC3335002646BF56B30600281577534A1
:100C5E0002D26043E680E52D54066026A840A941E5
:0F0C6E00C3E913F9E813F8C2AF53E67F7591009D
:100C7D00C3E498F594E499F595759104D26043E633
:100C8D0080D2AF22D265754400752000306B03759C
:100C9D002040020CB0D265754400752040306B03C6
:100CAD00752000D2AF7801206722E52D5406600231
:100CBD00C265C3E541940540137802940540087858
:100CCD0003940540027806306902780A206019E520
:100CDD0044601530690AC3E53394034003D53406E7
:100CED00D2AFD26CA18A915FD2AF0000C2AF2067A4
:100CFD0026E541C3FB940F40027B0FEB24053073B7
:100D0D000123306A02742820620123F930690279C7
:100D1D0082E58BC39940B50544E59E7005E59B02C0
:100D2D000D31E59A5440B52002A17430690A08C30B
:100D3D00E8940A40010881D920650281B0C265534B
:100D4D00E67F7591003067107594007595FE75916D
:100D5D0004D26043E68081B0AE40AF41C3E49EF55E
:100D6D0094E49FF595A15BC3E5339402500281B0E5
:100D7D0030650281B0D802A18881D9C26C53E67F5B
:100D8D00759100855494855595759104854E5685BC
:100D9D004F57D26043E680D2AFE52D540660082050
:100DAD006A020533020DC4306C0D206B0A206507F5
:100DBD001581158102163D227800306405306502DB
:100DCD007801E53775F007A4F9E5F028F5F0E9A20B
:100DDD00F013A2F113A2F213F537C39478500375F3
:100DED003778C3E53795384008D266C297C295C2A9
:100DFD0093306002A1FE855056855157D26043E66F
:100E0D008022207D14C2AF754302C294D296D2AF18
:100E1D00759F33759E00020FF0C2AF754302C294E9
:100E2D00D292D2AF759F33759E00020FF030724390
:100E3D00207D20C2AF75430390013D757E10C29396
:100E4D00C292306204D295C158D294D2AF759E220F
:100E5D00020FF0C2AF75430390013D757E10C2972E
:100E6D00C296306204D295C178D294D2AF759E23CA
:100E7D00020FF0207D17C2AF754303900118C29386
:100E8D00306202D295D2AF759E22020FF0C2AF75BD
:100E9D004303900118C297306202D295D2AF759E6E
:100EAD0023020FF0207D11C2AF754304C296D2927A
:100EBD00D2AF759E23020FF0C2AF754304C292D21A
:100ECD0096D2AF759E22020FF0307249207D23C25B
:100EDD00AF75430590012C757E40C295C29430626A
:100EED0004D297C1F4D296D2AF759F33759E00028E
:100EFD000FF0C2AF75430590014E757E04C295C2C9
:100F0D0094306204D293E117D292D2AF759F3375AC
:100F1D009E00020FF0207D1AC2AF75430590010EA1
:100F2D00C295306202D297D2AF759F33759E000283
:100F3D000FF0C2AF754305900122C2953062E8D221
:100F4D0093D2AF759F33759E00020FF0207D11C2B5
:100F5D00AF754306C292D294D2AF759E22020FF0A6
:100F6D00C2AF754306C296D294D2AF759E23020FBF
:100F7D00F0307242207D20C2AF75430190014E7555
:100F8D007E04C297C296306204D293E19CD292D273
:100F9D00AF759E23020FF0C2AF75430190012C7502
:100FAD007E40C293C292306204D297E1BCD296D2F7
:100FBD00AF759E22E1F0207D16C2AF754301900101
:100FCD0022C297306202D293D2AF759E23E1F0C256
:100FDD00AF75430190010EC293306202D297D2AF2A
:100FED00759E22C2662290010C757E00C297C29535
:100FFD00C293C296C294C292C262227880760708CA
:10100D0076070876010876040876FF0876FF0876DD
:10101D0008087602087601087601788C7601087644
:10102D00000876B40876FF0876FF0876FF08760389
:10103D000876FF0876010876FF0876250876D00831
:10104D0076780876C80876040876FF087601087663
:10105D000008767A08761008760108760108760081
:0F106D000876FF227887E6FFC2727888C27DE698
:10107C0030E102D27DC27E7889E630E102D27EC3B5
:10108C00EF94026008758E01D27302109E758E006B
:10109C00C273227880E6149000809378A4F678814D
:1010AC00E6149000809378A5F67886E61490008D6F
:1010BC009378A6F6789FE6F8700108C3E89411407F
:1010CC00027811E82828F56E256E256E28F56F2517
:1010DC006E2828F570789CE67538FF75390CB402CB
:1010EC00067538A075390AB403067538827539054A
:1010FC0078A3E61490009A93F569120FF3222278E4
:10110C0096E6FA7897E6FB7888E6B40305C3EB9489
:10111C000EFB307F047A007BFFC3EB9AFCC39482F6
:10112C0050027C827575000575EC8575F0A4C3E5DD
:10113C00F0947D40F222D27F310B12055C7A007B59
:10114C00007C10120552E55F2AFA74003BFBDCF3BD
:10115C007C04C3EB13FBEA13FADCF7FEC27F310B02
:10116C0022E5EF20E6037520000520903DFFE520E9
:10117C00146006901FFF1460009304600375EF1257
:10118C0053D9BF7581C043FF8012054D75EF0243E3
:10119C00B203E5B3240420E70DF521E5B120E00608
:1011AC008521B343B101120FF375800875A4007546
:1011BC00F1FF75D4F775900275A5FC75F2FD75D528
:1011CC000075A0FF75A60075F30075D60075B0FF0D
:1011DC0075A70175F4FF75E241E4F8F6D8FD756B5F
:1011EC0001110812168578988676753001C2AF12F7
:1011FC00056612057612055C12057D12055C12055A
:10120C008412055C1217A712056612056612056199
:10121C00C2AF78FA79FA308307D9FBD8F7021C00F1
:10122C001171119F310A310B78988676120FF37574
:10123C00885075891275C82475910475D84075A8A5
:10124C002275B80275E690759B80759D00759A8025
:10125C00759C0075D10E75BC5875BB0175BA1F75A0
:10126C00E88012054DD2AF1208A553DACF207E03C9
:10127C0043DA20307E0343DA1043DA01C2D8C2715C
:10128C00120566D2617B037A0CE55E70077A0CDB83
:10129C000302121C12055C20700302121CC270E5C2
:1012AC005FC3940240E1E52F541F856160F561B581
:1012BC0060D5DAD5C26153DACF207E0343DA203011
:1012CC007E0343DA10C2D8C27178A2E67008D274D9
:1012DC00E52F54E0F52FC2757529001205613074A5
:1012EC0009C3E529940A4002D275120552780230DE
:1012FC0074027800C3E55F9840F0C2AF1205761215
:10130C000576120576D2AF120566754D00120552A0
:10131C00788CE6C3940150030213EFE530C39401BB
:10132C0050030213EF207435C3E55F94FF500302A2
:10133C0013EFC2AF12058BD2AF120561C3E55F94F8
:10134C000150EFC2AF120576120557120576D2AFD7
:10135C00120561C3E55F94FF40E902182C7F05D2AA
:10136C007F310B120561C2AFC27F310BAE5FC3E59B
:10137C005F947FD2AF407612054DC2AF12058BD26F
:10138C00AFDFDC3142C3EE94057897F61205661296
:10139C0016C61217AF7F0AD27F310B120561C2AF8E
:1013AC00C27F310BAE5FC3E55F947FD2AF50E612C4
:1013BC00054DC2AF120576120557120576D2AFDF76
:1013CC00D63142EE24057896F61205661216C61230
:1013DC0017DE120561310BC3E55F94FF50026131DA
:1013EC0002182CC3E55F954D4003855F4D120561D6
:1013FC0078017988E7B403027805C3E55F98400269
:10140C006119C2AF12058B12058B12058BD2AF126C
:10141C000566753000E4F531F5320531E531F470CF
:10142C00390532789AE67819146012783214600D06
:10143C00787D14600878FA146003753200C3E532C5
:10144C0098401715327531B478998676C2AF12056B
:10145C008BD2AF78988676120561120557E52A7003
:0E146C0005307402411C78012074027806C31A
:10147A00E55F9840A7120561E52A700302121CC2B3
:10148A00AF120FF3E4F522F523F524F525F526F539
:10149A006AD2AF7885E6C333F568E4F545F546F5D3
:1014AA0047F548F549F573F52CF52DF537757308A9
:1014BA0075BB1E12054D120938E5E820ECFBA8BDE4
:1014CA00A9BEE97001F8887412093C75730875BBE6
:1014DA001E7887E6FE760211717887EEF6C2AF753E
:1014EA0064FF1209F7852264852265852266D2AFD8
:1014FA0075220175240175250175260185636C75B0
:10150A006D017888E6B40307C27D307602D27DD2B7
:10151A0068D269753300120F59120F7E120A171218
:10152A000A1E120A17120A1E120A17021544C2AF1D
:10153A001171D2AF75730075BB01120CA212065657
:10154A00120DC5120E0F120A1E120C91306D0312E3
:10155A0006F620670312084830670312088F120D37
:10156A00C5120E3A120A1E120CA2306D031207326D
:10157A00120DC5120EB1120A1E120C91306D031211
:10158A000790120DC5120ED6120A1E120CA2306D49
:10159A00031207ED120DC5120F59120A1E1209384D
:1015AA00120C91120DC5120F7E12093C120A1E303E
:1015BA00692F206B2C85676485676585636C756DFB
:1015CA000179187A0CC3E533994009C269D26A8A4B
:1015DA00350215EBC3E55F94014003021544021678
:1015EA0045306A1B206B18E535147004C26AA138AD
:1015FA00F535C3E55F9401400302154402164575AB
:10160A003600C3E5629401400985676585636C7598
:10161A006D01C3E56278FA985021307404E52A60B6
:10162A001A78F0306B058567647820C3E5419850D5
:10163A0002A1440536E55F6002C148753600C2AFB3
:10164A00120FF37887E6FE760211717887EEF6E4D8
:10165A00F522F523F524F525F526F568C268D2AFFB
:10166A0012054D120FF3307406E52A7002411C78F8
:10167A008DE6C39401400241F68121901A0D78202B
:10168A00121708E520B4A50CA3121708E520B45ACE
:10169A00030216A611081216C60216C5901A037876
:1016AA00807B0A121708A308DBF9901A0F788C7B43
:1016BA0018121708A308DBF9901A2722C2AF1217CB
:1016CA0047121721901A00740E12170DA3740412F0
:1016DA00170DA3741412170D901A0378807B0A123F
:1016EA00170CA308DBF9901A0F788C7B1812170CC9
:1016FA00A308DBF912175A121738901A2722E49313
:10170A00F622E6438F01538FFD75EF0275B7A57573
:10171A00B7F1F0538FFE22438F02438F0175EF0218
:10172A0075B7A575B7F1901A0DF0538FFC22901A70
:10173A000D74A5F10D901A0E745AF10D227A3079B2
:10174A00D07820901A40F108E520F709A3DAF722A9
:10175A007A3079D0901A40E7F10D09A3DAF922AB71
:10176A0077A878BB01027980BB02027981BB0302A8
:10177A007982BB04027994BB05027983BB0602799C
:10178A0086BB07027992BB08027987BB0902799C5A
:10179A00BB0A027988BB0B027989E8F7227C051219
:1017AA000566DCFB22C2AF12057612057D1205849E
:1017BA0012058B12055712057612057D1205841241
:1017CA00058B12055712057612057D12058412053E
:1017DA008BD2AF22C2AF12058B12058412057D127D
:1017EA00057612055712058B12058412057D12051E
:1017FA007612055712058B12058412057D1205769D
:10180A00D2AF22AE77AF78C2AF1205761205761242
:10181A000576120557DEF212058B120557DFF8D24C
:10182A00AF221217AF1217A71217A775770175788B
:10183A0001757900110D7C05AD5F120566C3ED9542
:10184A005F70F5C3E55F9401400AC3E55F94FF400A
:10185A003702186F1217691216C61217AFC2AF7580
:0E186A00EF121217A7DCD10579C3E5799403BC
:10187800500280C21217A70578E5771490009F934D
:10188800F808C3E57898500280A91217A71217A77D
:101898000577C3E577940C5002809512100812164C
:0918A800C6C2AF75EF121217A7BA
:0319FD0002116D67
:101A00000E041407070104FFFF08020101A55A0193
:101A100000B4FFFFFF03FF01FF25D078C804FF01DA
:081A200000FF10010100FFFFAF
:101A4000235467794B4637304148562320202020C5
:101A500023424C48454C4923463331302320202033
:101A60002020202020202020202020202020202076
:101C0000C2AFC2D353D9BF7581C043B20343FF8073
:101C1000752438752503B1C975EF0275E24043F1AB
:101C20000853A4F775D400D2837DFA780379E67C53
:101C300010752200752300901DD67B0675249875BB
:101C400025013083028142208308D8FBD9F9DCF7D3
:101C500081B4308308D8FBD9F9DCF781B4B189E4C9
:101C600093A3C39A6004DDC381B4DBDBB17B600264
:101C7000812B7B08E493FAA3B15CDBF87A30B15C8A
:101C8000752200752300B17BEAFCEBFDC3ED94FEE9
:101C9000400EB17B8A278B28ED30E0048A828B834B
:101CA000B17B7AC270D8C3ED94FE601350CEBD00F4
:101CB00025EC60097520007521FF0200008100A855
:101CC00027A9280809D804D90281D3B17FEA89AAB3
:101CD000F281C50D81A0C3ED94035049EDA2E092BD
:101CE000007AC5C3E5829400E583941C50902000DF
:101CF00010438F02438F0175B7A575B7F1F030001F
:101D00001FA827A9280809438F01538FFDD804D99C
:101D100002A12089AAE275B7A575B7F1F0A3A10DBC
:101D2000538FFC817C7AC1BD030CE493A3FAB140CC
:101D3000DCF8B138817C817EAA22AB23B15CEBFA5E
:101D4000EA6222752608C3E52313F523E52213F57D
:101D50002250066323A0632201D526EAB1C9B1C986
:101D600075260AEAF4200102D283300102C283B14F
:101D7000C9C3134002C201D526EB22B17FEAFB2082
:101D80008302A17F308302A184752608AE24AF258B
:101D9000C3EF13FFEE13FEB1CDB1C9C3EA13308315
:101DA000024480FA30E703632201C3E52313F523DD
:101DB000E52213F52250066323A0632201D526D91C
:101DC000E52265236523F52222AE24AF250E0FDE22
:101DD000FEDFFCD20122424C48656C693437316326
:041DE000F3100601F5
:00000001FF
